:020000021000EC
:10F800000C9446FC0C9463FC0C9463FC0C9463FC19
:10F810000C9463FC0C9463FC0C9463FC0C9463FCEC
:10F820000C9463FC0C9463FC0C9463FC0C9463FCDC
:10F830000C9463FC0C9463FC0C9463FC0C9463FCCC
:10F840000C9463FC0C9463FC0C9463FC0C9463FCBC
:10F850000C9463FC0C9463FC0C9463FC0C9463FCAC
:10F860000C9463FC0C9463FC0C9463FC0C9463FC9C
:10F870000C9463FC0C9463FC0C9463FC0C9463FC8C
:10F880000C9463FC0C9463FC0C9463FC11241FBE69
:10F89000CFEFD0E1DEBFCDBF11E0A0E0B1E0E0E00E
:10F8A000F0E002E00BBF02C007900D92A030B1075C
:10F8B000D9F712E0A0E0B1E001C01D92A434B10775
:10F8C000E1F70C94C4FF0C9400FC0F93EF93FF93AB
:10F8D00040D0FC01062F36D0FF91EF910F91089593
:10F8E0000F930F921F92EF93FF9333D0FC010B0104
:10F8F00001E028D0FF91EF911F900F900F91089594
:10F900000F930F92EF93FF9324D0FC0160FD60935F
:10F910006800D895802DE395D895902DFF91EF91B3
:10F920000F900F9108950F930F9213D0082E09E0B6
:10F9300009D00F900F9108950F930BD001E102D0E1
:10F940000F910895E199FECF00936800E895FFFFBD
:10F9500000000091680000FDFCCF089583E08093D3
:10F96000990080919A00806180939A0080919A001A
:10F97000886080939A00089580919C00992708954B
:10F9800040E050E04817590750F42AE633E0000001
:10F990002150304037FFFBCF4F5F5F4FF3CF0895CB
:10F9A00080919B00992780789070089580919A00AB
:10F9B0008F7E80939A0080919A00877F80939A002F
:10F9C00008950E94D6FC0C940000089580939C003A
:10F9D00080919B0086FFFCCF80919B008064809388
:10F9E0009B0008950E94D0FC8823E1F30E94BCFC98
:10F9F000803219F481E090E0089585E10E94E6FCF0
:10FA000080E090E008950895EF92FF920F931F9386
:10FA1000CF93DF937B01C0E0D0E0C617D70770F427
:10FA20008C010E94D0FC8823E1F30E94BCFCF80109
:10FA300081938F012196CE15DF0598F381E090E048
:10FA4000DF91CF911F910F91FF90EF90089590E07B
:10FA5000282F33272138310589F02238310524F445
:10FA60002038310549F00DC02238310549F02839D8
:10FA7000310539F493E005C092E003C091E001C084
:10FA800092E1892F9927089540E050E0609140016C
:10FA90007091410146175707E8F4E2E4F1E08091E4
:10FAA00042028EBB8091420290914302292F33275C
:10FAB0002FBB0196909343028093420280818DBBBD
:10FAC000E29AE19AE199FECF4F5F5F4F3196461778
:10FAD000570728F308950F931F93CF93DF938091D7
:10FAE00042029091430297FF03C081E08BBF01C0A7
:10FAF0001BBE00E010E08091400190914101081789
:10FB00001907D8F4C2E4D1E08091420290914302F7
:10FB1000880F991F60E0800F911F0E9480FC8883EE
:10FB2000892F992789830E5F1F4F2296809140016C
:10FB3000909141010817190738F3DF91CF911F9178
:10FB40000F91089580914001909141010097C1F07B
:10FB5000E2E4F1E0AC01809142028EBB809142026E
:10FB600090914302292F33272FBB01969093430294
:10FB700080934202E09A8DB381934150504059F7EF
:10FB800008950F931F93CF93DF938C016115710537
:10FB900041F0EB01F80181918F010E94E6FC219771
:10FBA000C9F781E090E0DF91CF911F910F91089507
:10FBB0000F931F93CF93DF93C0E0D0E00FEF11E0DE
:10FBC000D0934302C0934202D7FF03C081E08BBFB2
:10FBD00001C01BBE809142029091430263E0880FF6
:10FBE000991F0E9465FC01501040C058DF4F17FF5D
:10FBF000E7CF0E949CFCDF91CF911F910F91089558
:10FC0000EF92FF920F931F93CF93DF938091420265
:10FC10009091430297FF03C081E08BBF01C01BBEE0
:10FC200000E010E080914001909141010817190710
:10FC300008F048C0EE24FF24E801CD5BDE4FF80158
:10FC4000EE5BFE4FEE0DFF1D4081888122969927C5
:10FC5000382F2227240F311D8091420290914302B8
:10FC6000880F991FB9018E0D9F1D0E9470FC82E0C4
:10FC700090E0E80EF91E9FEFE916F10401F3F8F2A7
:10FC80008091420290914302880F991F63E0800F98
:10FC9000911F0E9465FC8091420290914302880F5F
:10FCA000991F65E0800F911F0E9465FC0E949CFCDB
:10FCB00000501F4F80914001909141010817190792
:10FCC00008F4B8CFDF91CF911F910F91FF90EF9083
:10FCD0000895CF93C0E069E081E090E00E9480FC4D
:10FCE00084FF03C08F7E0E9493FC0E94D0FC882377
:10FCF000E1F30E94BCFC992782359105DCF4803544
:10FD000091050CF054C08134910509F45AC0823435
:10FD100091053CF48033910509F449C0C19759F12C
:10FD20002FC18234910509F45FC08534910509F42F
:10FD30005EC026C18635910509F4EDC08735910571
:10FD40004CF48235910509F461C08535910509F4BB
:10FD500065C016C18437910509F4A0C085379105A7
:10FD60002CF48436910509F472C00AC185379105D7
:10FD700009F4C1C005C10E94F2FC882309F4B5CF83
:10FD800084E10E94E6FC81E40E94E6FC86E50E9494
:10FD9000E6FC82E50E94E6FC80E20E94E6FC83E548
:10FDA0000E94E6FC84E50E94E6FC8BE406C00E940B
:10FDB000F2FC882309F499CF84E10E94E6FC80E1FB
:10FDC000E0C061E070E080E091E00E9404FD0E94EC
:10FDD000F2FC882309F489CF84E10E94E6FC80913B
:10FDE00000010E9427FDE9CF64E170E00AC061E0F4
:10FDF00070E080E091E00E9404FD8091000199276D
:10FE0000BC0180E091E00E9404FDD1CF0E94F2FC91
:10FE1000882309F46ACF0E94D8FDCECF62E070E05B
:10FE200080E091E00E9404FD0E94F2FC882309F426
:10FE30005CCF20910001809101019927982F88279C
:10FE4000820F911D9093430280934202B5CF63E0ED
:10FE500070E080E091E00E9404FD2091010180911A
:10FE600000019927982F8827820F911D90934101B7
:10FE700080934001BC0182E491E00E9404FD0E9455
:10FE8000F2FC882309F431CF80910201863419F401
:10FE90000E9400FE91CF0E9444FD8ECF63E070E08F
:10FEA00080E091E00E9404FD209101018091000119
:10FEB0009927982F8827820F911D90934101809355
:10FEC00040010E94F2FC882309F40FCF80910201C7
:10FED000863419F40E946BFD02C00E94A2FD84E1E9
:10FEE0000E94E6FC609140017091410182E491E042
:10FEF0000E94C1FD64CF0E94F2FC882309F4F5CE74
:10FF000084E10E94E6FC8EE10E94E6FC87E90E9403
:10FF1000E6FC82E052CF64E070E080E091E00E9475
:10FF200004FD0E94F2FC882309F4DFCE84E10E94E4
:10FF3000E6FC80910001803531F480910101882335
:10FF400061F4C82F17C0883531F4809101018830E1
:10FF500061F4C3E00FC0803531F480910101883035
:10FF600049F4C2E007C0883529F480910101882353
:10FF700009F4C1E069E08C2F99270E9480FC1DCF15
:10FF800085E10E94E6FCB1CECFEFD0E1DEBFCDBF70
:10FF9000CEE1F8948EEF9FE00E94F7FF843B61F47E
:10FFA0008FEF9FE00E94F7FF833C31F48DEF9FE0DD
:10FFB0000E94F7FF80936F000E94AEFC0E94BCFC81
:10FFC00084E690E00E94C0FC0E94D0FC882321F4CB
:10FFD000C150C8BBCC23A1F7CC2319F00E9469FE05
:10FFE00002C00E94E1FC80E090E00C94FFFFE199E8
:10FFF000FECF9FBB8EBBE09A99278DB30895FFCFAC
:040000031000F800F1
:00000001FF
